:0200000480007A
:100000006F008004732F2034930F80006308FF0378
:10001000930F90006304FF03930FB0006300FF038E
:10002000130F000063040F0067000F00732F2034CC
:1000300063540F006F00400093E19153171F0000BD
:1000400023223FFC6FF09FFF93000000130100008C
:10005000930100001302000093020000130300004C
:100060009303000013040000930400001305000034
:10007000930500001306000093060000130700001C
:100080009307000013080000930800001309000004
:1000900093090000130A0000930A0000130B0000EC
:1000A000930B0000130C0000930C0000130D0000D4
:1000B000930D0000130E0000930E0000130F0000BC
:1000C000930F0000732540F16310050097020000B4
:1000D000938202017390523073500018970200000F
:1000E00093824202739052309B021000939252030B
:1000F0009382F2FF7390023B9302F0017390023AF5
:100100007350403097020000938242017390523046
:10011000735020307350303093010000970200007C
:10012000938282EE73905230130510001315F5017F
:10013000635C05000F00F00F930110009308D005D9
:10014000130500007300000093020000638A0200A0
:1001500073905210B7B200009B82921073902230BD
:100160007350003097020000938242017390123462
:10017000732540F1730020309300400113016000AB
:100180003BF7200293032000930120006314770CB7
:100190009300C0FE130160003BF720029303200090
:1001A000930130006318770A930040011301A0FF08
:1001B0003BF720029303400193014000631C770842
:1001C0009300C0FE1301A0FF3BF720029303C0FE83
:1001D0009301500063107708B700008013011000EE
:1001E0003BF720029303000093016000631477063D
:1001F000B70000801301F0FF3BF72002B703008037
:100200009301700063187704B700008013010000A9
:100210003BF72002B703008093018000631C770244
:1002200093001000130100003BF72002930310001D
:100230009301900063107702930000001301000007
:100240003BF72002930300009301A00063147700A2
:10025000631030020F00F00F6380010093911100D2
:1002600093E111009308D00513850100730000008D
:100270000F00F00F930110009308D0051305000044
:1002800073000000731000C00000000000000000B8
:10029000000000000000000000000000000000005E
:1002A000000000000000000000000000000000004E
:0C02B00000000000000000000000000042
:1010000000000000000000000000000000000000E0
:1010100000000000000000000000000000000000D0
:1010200000000000000000000000000000000000C0
:1010300000000000000000000000000000000000B0
:081040000000000000000000A8
:040000058000000077
:00000001FF
